:020000040000FA
:1000000000400110210100002D010000310100001D
:1000100000000000000000000000000000000000E0
:10002000000000000000000000000000350100009A
:100030000000000000000000390100002501000060
:100040003D010000410100004501000049010000A0
:100050004D01000051010000550100005901000050
:100060005D010000250100002501000000000000E6
:100070000000000000000000000000000000000080
:1000800000000000250100002501000025010000FE
:1000900025010000250100002501000025010000C8
:1000A00025010000250100002501000025010000B8
:1000B00025010000250100002501000025010000A8
:1000C0000448854601F09AFA0048004709010000FB
:1000D000C046C0460040011008B5C021172000F0FE
:1000E0001BFC0521684601700021417000F0CDFC29
:1000F00008BD10B50024FF20F53000F00AFF0520F0
:1001000000F024FD044610BD00F0D5FDFFF7E4FF2C
:1001100005E0FF20F53000F0FCFEFFF7EAFFF8E70E
:1001200001480047FEE70000C100000000BFFEE7F5
:1001300000BFFEE700BFFEE700BFFEE700BFFEE72F
:1001400000BFFEE700BFFEE700BFFEE700BFFEE71F
:1001500000BFFEE700BFFEE700BFFEE700BFFEE70F
:10016000FEB505460C4600200190002600900027B1
:100170000120F749C8700846407C80218843F44933
:100180004874002C04D1F34A2B21F3A001F069F943
:10019000002D06D0012D04D0EE4A2C21EEA001F056
:1001A00060F92068002803D0F8492068884204D903
:1001B000E84A2D21E8A001F054F9A088002807D0D2
:1001C000A088042804D0E34A2E21E3A001F049F9D5
:1001D000E088002807D0E088082804D0DD4A2F21D5
:1001E000DDA001F03EF92089002807D020890228EF
:1001F00004D0D84A3021D8A001F033F960894028D2
:1002000007D06089002804D0D24A3121D2A001F061
:1002100028F9A089002807D0A089102804D0CD4A49
:100220003221CDA001F01DF9E089002804DDE0892C
:10023000FF210131884204DDC64A3321C6A001F006
:1002400010F9208A002804DD208AFF21013188422C
:1002500004DDC04A3421C0A001F003F9208829013F
:10026000CB4A5052002D12D1CA4E290189180E8155
:10027000E0898019290189184881C74E2901891808
:100280004E80208A801929018918888012E0C34E87
:100290002901BF4A89180E81E0898019290189182E
:1002A0004881BF4E290189184E80208A8019290172
:1002B00089188880A07A217B0843217A0843A17994
:1002C00008432179084381210843C0B201902901E4
:1002D000AF4A891801988873002D04D1B148009065
:1002E0009B4F123704E0AF4811300090984F3237DF
:1002F00001210907009840180078410849000122AF
:1003000012070098801801702801A14A115A384636
:1003100000F014FA28019E4A8018018938460830F6
:1003200000F00CFA28019A4A8018418938460A30B0
:1003300000F004FA2801964A8018018938460C30EA
:1003400000F0FCF92801924A80184188B81C00F09E
:10035000F5F928018E4A80188188381D00F0EEF9E1
:1003600028018B4A80184188B81D00F0E7F9012167
:1003700009070098401800782901854A8918897B67
:10038000084301221207009989180870FEBD10B5B4
:100390000446002C06D0012C04D0834A71216EA0A3
:1003A00001F05FF8002C0BD1694820300078012162
:1003B00008436749203108700846007808700AE051
:1003C00063482030407C0121084361492031487452
:1003D0000846407C487410BDF8B504460F46002519
:1003E0000026002C06D0012C04D0704A99215AA076
:1003F00001F037F8002C02D1554D123501E0544D73
:10040000323528460830002804D1684AA02152A07D
:1004100001F027F8002C09D100BF6548807B6449B2
:10042000C97B090208430028F7DC0AE000BF6048E6
:100430004030807D5E494031C97D09020843002873
:10044000F5DC28460C3000F082F906465948301891
:10045000077028460A3000F07AF9B04205D12846E4
:10046000083000F074F9064601E0701C86B231468F
:1004700028460C3000F062F9F8BDF8B504460025B6
:1004800000260027002C06D0012C04D04A4AB921AE
:1004900031A000F0E6FF002C02D12D4D123501E015
:1004A0002B4D3235A81D00F052F906464148301850
:1004B00000F04DF90746281D00F049F9B04204D17B
:1004C000A81C00F044F9064601E0701C86B23146D3
:1004D000A81D00F033F93846F8BD10B50446002CCD
:1004E00006D0012C04D0354ACC211BA000F0B9FF66
:1004F000002C04D12E48123000F029F910BD2C48F0
:100500005A3000F024F9F9E7F7B584B004461546EF
:10051000002003900026002702900190002C06D0B6
:10052000012C04D0264ADC210BA000F09AFF05988C
:10053000002804D1224ADD2107A000F092FF002C00
:1005400040D10348123001901948123002903DE02A
:1005500040800010601600002E2E5C2E2E5C2E2E89
:100560005C2E2E5C4C69627261726965725C6472A9
:1005700069766572735C756172745C796331317828
:10058000785F756172742E630000000010A7000090
:100590001405011034050110340601103407011050
:1005A00034080110608000006B160000781600000F
:1005B000008300100000011087160000991600004B
:1005C000AA1600005848019058480290029800F07E
:1005D000BEF80390002D06D00398A84202DA00204E
:1005E00007B0F0BD03950398002800D1F8E7019803
:1005F000801D00F0ACF80646002714E04C48301887
:1006000001780598C1550198001D00F0A0F8B0428E
:1006100005D10198801C00F09AF8064601E0701C94
:1006200086B2781C87B203988742E7DB314601988F
:10063000801D00F083F83846D2E7F7B582B0044653
:100640000026002001900025002C07D0012C05D0A9
:10065000384AFF210331384800F003FF039800288F
:1006600005D1344AFF210431334800F0FAFE0498E2
:10067000002805DC2F4AFF2105312F4800F0F1FE4C
:10068000002C02D1284D203D00E0274D284608309F
:10069000002805D1274AFF210C31274800F0E1FE50
:1006A000002C0BD100BF21485A38807B1F495A3992
:1006B000C97B090208430028F5DC0AE000BF1B489B
:1006C0001A38807D19491A39C97D09020843002862
:1006D000F5DC28460C3000F03AF80646002718E012
:1006E0000398C05D12497118087028460A3000F05E
:1006F0002EF8B04205D12846083000F028F806460A
:1007000001E0701C86B20198401C80B20190781CF8
:1007100087B204988742E3DB314628460C3000F06C
:100720000DF8019805B0F0BD728000105A830010DA
:1007300000000110BF1600005805000070B5044607
:100740000D46257000F059F82812607070BD70B524
:1007500004460025002600F050F8257800F04DF8FA
:1007600066783002FF21090208400543284670BD23
:1007700070B50446002500F040F8257800F03DF8FB
:1007800060780002054300F038F8A07800040543C3
:10079000284670BD10B503E00B780370491C401C5F
:1007A0001346541EA2B2002BF6D110BD0146002202
:1007B00001E0521C491C08780028FAD190B2704719
:1007C00000BFFEE710B5002106E00F4A00BF134648
:1007D000521E002BFBD1491C8142F6DB10BD10B527
:1007E000002107E07D22120100BF1346521E002B9C
:1007F000FBD1491C8142F5DB10BD00BF00BF00BF2B
:1008000000BF00BF70470000204E000070B50446D6
:100810000D4600F005F9202C00D170BD002D02D04E
:10082000012D12D108E03E20E106C90E7F4A891849
:1008300052058918087009E03F20E106C90E7B4A7D
:10084000891852058918087000E000BF00BF00F049
:10085000E7F800BFE1E770B504460D4600F0E0F8A8
:10086000202C00D170BD012D06D0022D0DD0032DFE
:1008700014D0042D24D11AE00020E106C90E6B4AE1
:1008800089185205891808701BE04020E106C90E3E
:10089000664A891882058918087012E08020E106EE
:1008A000C90E624A891842058918087009E0C020FB
:1008B000E106C90E5D4A891852058918087000E0E2
:1008C00000BF00BF00F0ACF800BFCBE730B5014679
:1008D000202900D130BDCB06980F4A07520F03469E
:1008E000AB33012424071B191C78012393409C433C
:1008F0000346AB3301252D075B191C700346AF334C
:100900002C461B191B7801249440A3430446AF34A2
:100910006419237000BFDDE7C206D20E434BD21824
:100920005B05D2181170704770B502460023002491
:10093000002553075B0FD006840F081901263607E0
:100940003043057801209840284070BD10B504461A
:10095000202C01D1FFF734FFE006C00E3449FFF729
:10096000E3FF10BD70B502460B46202A00D170BDD2
:10097000D406A00F5107490F002B02D0012B3AD10A
:100980001CE00446AB3401252D07641924780125A9
:100990008D402C43E5B20446AB3401263607A4193A
:1009A00025700446AF3435466419257801248C40FF
:1009B000A5430446AF34A41925701CE00446AF34A7
:1009C00001252D076419247801258D402C43E5B2BB
:1009D0000446AF3401263607A41925700446AB340B
:1009E00035466419247801258D40AC430546AB3566
:1009F000AD192C7000BF00BF00BFB8E770B504464A
:100A00002046FFF7A3FF0546002D04D00021204615
:100A1000FFF7A8FF03E001212046FFF7A3FF70BD09
:100A200000BF00BF00BF00BF00BF70478080000054
:100A30001C830000FFB589B0129E7D21C900099872
:100A400048430B99441AE717079706940B990A989D
:100A5000401A05900C98851B0495049DE817079F84
:100A6000069C0890204639462A46089B00F048FD1F
:100A7000019100900598C3170246009800F01AFDF6
:100A80008019039003980DB0F0BD10B5044620788E
:100A9000002819D02078012816D02078022813D0F9
:100AA0002078032810D0207804280DD0207805283D
:100AB0000AD02078062807D02078072804D0684A72
:100AC000212168A000F0CDFC607800280DD060786E
:100AD00001280AD06078022807D06078032804D063
:100AE0005F4A22215FA000F0BCFC607800018F21EA
:100AF0000843674948747C20654960398871AA2099
:100B0000634988742078302108436149C874802083
:100B10006049C87010BD01465F4A7C205C4B603B59
:100B20009871AA205A4B987430200843D8748020BA
:100B3000584BD87000BF1046521E0028FBD15748B2
:100B4000807C564BDB7C1B0218437047F1B58AB0A2
:100B50000020099008900790FF26F53677000024C2
:100B600000254B48407C7021084000110690002071
:100B700002900390049005900E2202A9484800F0CC
:100B80008CFA6946487D0002097D08434549884240
:100B900002D0601E0BB0F0BD0698002804D00228D9
:100BA00019D0032845D12DE06846407A01026846F5
:100BB000007A08437D21C900484304466846C07B4B
:100BC00000026946897B08437D21C90048430546E8
:100BD0004E100F4630E06846C07A01026846807ABF
:100BE00008437D21C900484304466846407C000212
:100BF0006946097C08437D21C900484305462A4EC1
:100C0000254F19E06846407B01026846007B084397
:100C10007D21C900484304466846C07C00026946FD
:100C2000897C08437D21C900484305461E4E1F4F5D
:100C300002E00020C043ADE700BF002C01D0002D32
:100C400002D10020C043A5E70A98FFF764FF09908E
:100C50003B462246294600960998FFF7EBFE99E7A6
:100C6000D61600002E2E5C2E2E5C2E2E5C2E2E5CB8
:100C70004C69627261726965725C647269766572F0
:100C8000735C6164635C4472765F6164632E6300CD
:100C900060890010608000108813000040830010FD
:100CA000E21F000055AA0000B80B0000E40C000091
:100CB00000BF00BF704710B5B648B74908600020B4
:100CC00009680861B548B4490968C8600120B2499B
:100CD000096808720020B04909680860B04C601EBD
:100CE000B049884200D90CE0601EAF494861032139
:100CF000081F00F017F90020AB4988610720086140
:100D000000BF10BD0246002A00D17047A24801680A
:100D100004E08A4201D10120F7E709690869002847
:100D2000F7D100BFF1E7F0B504460D461646002C9A
:100D300000D1F0BD2046FFF7E5FF002801D00120DB
:100D4000F7E7002B02D19548E06000E0E36072B65F
:100D50006560964800684019206001202072667224
:100D60008D48076804600068076162B60120E0E70B
:100D70000146002900D170478748026809E0914286
:100D800006D18A4B48681B68C01808600120F2E74A
:100D9000126910690028F2D100BFECE700217E4AF9
:100DA000106801E0491C00690269002AFAD1704705
:100DB00010B50246002A00D110BD7648824201D10A
:100DC0000020F9E7744801680B460FE08A420BD116
:100DD000002008728B4203D16F4C0869206001E04B
:100DE000086918610120E7E70B46096908690028CE
:100DF000ECD100BFE0E710B56D480078002820D0A6
:100E000000206B4908706448046817E0207A0128C4
:100E100013D166492068096888420ED8607A002894
:100E200003D12046FFF7C4FF04E060496068096809
:100E300040182060E16860698847246920690028BB
:100E4000E4D110BD5449086802E000210172006934
:100E500001690029F9D14F494F4A11607047554A3D
:100E60001278544B5B781B021A43524B9B781B043D
:100E70001A43504BDB781B061A43104600214E4A9A
:100E80001268002A02D14C4A10601AE04A4A1268DD
:100E9000824202D9484A10607047474A1268811A54
:100EA0000DE0424A1268521C404B1A60424A1268D6
:100EB0002032414B1A60203901223D4B1A70202903
:100EC000EFD200BFE8E700B5FFF7C9FF01203849BE
:100ED000087000BD70B5034600BF334E7569182613
:100EE0005E4334460022304EB1690FE02E4EB069A9
:100EF00088420BD0884202D20E1AB21802E02E1A93
:100F00007618B2180146A24200D300E0EEE700BF17
:100F100070BD10B504467D21C90061430846FFF746
:100F2000D9FF10BD10B5002819DA244A03071B0F9A
:100F3000083B9B089B00D2588307DC0EFF23A3408D
:100F40009A438B071B0E8407E40EA3401A431B4BE6
:100F50000407240F083CA408A4001A5118E0184AFA
:100F600003231B02D21883089B00D2588307DC0E90
:100F7000FF23A3409A438B071B0E8407E40EA34074
:100F80001A430F4B032424021B198408A4001A518E
:100F900010BD00003409011000050110B10C000063
:100FA000C05D0000FFFFFF0000E000E0040501104D
:100FB00008050110008300100C0501101CED00E075
:100FC00000E100E04948C07C402188434749C8749B
:100FD000704710B54548C07C402108434349C87458
:100FE000FF202D30FFF776FF10BDC00000BF404A44
:100FF00010710104090E517100BF002191717047F9
:1010000010B582203A49C8710120FFF763FF8020A4
:101010003749C8718220C8710D20FFF75BFF10BDF2
:1010200070B505460C46FFF7EBFFA2203049C871AA
:1010300000BF0D722804000E487200BF00BF8C7202
:101040002004000EC87200BF1120887101202849B9
:101050004039887270BD70B506460D46144630465C
:10106000FFF7C3FF21462348FFF7DAFF00BF2248FE
:10107000007C022108400028F9D083201C49C87157
:10108000002007E01B49411801221207114309788B
:101090002954401CA042F5D370BDF7B5144672B672
:1010A0000026002700256709E006C00E002800D0B2
:1010B0007F1CFFF78EFF002612E0202C01D9202094
:1010C00000E020460546224601990098FFF7C3FF3D
:1010D000009840190090019840190190641B761CFB
:1010E000BE42EAD3FFF76EFF62B6FEBD6089001014
:1010F00040800010234C00002083001000B585B014
:10110000D94800900021684681818180C180418159
:101110000181FF210131C1810182D448007800287A
:101120000AD1D24988780821FFF7F6FBCF494878E1
:101130000921FFF7F1FB0DE0CC480078012809D127
:10114000CA4988780C21FFF7E7FBC84948780D2188
:10115000FFF7E2FBC54908786946FFF701F805B0DB
:1011600000BDC249087070470178C04A117081788B
:10117000917041785170704770B504460D46AAB21F
:10118000BA4908782146FFF758FA70BD0FB4F0B598
:101190008BB011A8019042E1002400E0641C10987B
:1011A000005D252803D01098005D0028F6D1002CA2
:1011B00003D021461098FFF7DFFF10980019109018
:1011C000109800782528E6D11098401C1090002532
:1011D0002020039000BF10980178401C10903829FF
:1011E00030D014DC332928D008DC25296FD03029F1
:1011F00020D031291FD032296AD11DE034291DD0D9
:1012000035291CD036291BD03729F5D119E0702992
:1012100073D008DC392916D0582970D0632922D020
:101220006429E9D12AE073293CD075295AD078295C
:10123000E2D171E000BF00BF00BF00BF00BF00BF30
:1012400000BF00BF00BF10982038C07F302802D1F7
:10125000002D00D103900A20454310982038C07F0C
:1012600030384519B7E7019800680A900198001DC9
:10127000019001210AA8FFF77FFFCFE001980068E5
:101280000A900198001D019000260A98002805DAAE
:101290000A9840420A900120099001E0002009903C
:1012A0000A2747E00198006808900198001D019006
:1012B000002400E0641C0898005D0028FAD1214653
:1012C0000898FFF759FFA5420BD92D1B05E09AE0BE
:1012D0009FE0012166A0FFF74FFF28466D1E002802
:1012E000F7D19BE0019800680A900198001D0190D9
:1012F00000260A27002009901CE00EE0FFE7019875
:1013000000680A900198001D019000261027002017
:101310000990582002900DE000BF019800680A90E3
:101320000198001D019000261027002009907820C8
:10133000029000BF012403E02046784304466D1E5E
:10134000204678430A99884207D8214679430846BF
:10135000394600F099F8A042EED00998002800D054
:101360006D1E0998002809D00398302806D12D2237
:101370003046761C04A90A5400200990012D0BD98F
:10138000102D09D26D1E05E03146761C04AA039883
:1013900050546D1E002DF7D10998002804D02D223D
:1013A0003046761C04A90A5426E0029878280FD10A
:1013B00021460A9800F068F83946009000F064F879
:1013C0002C480068425C3046761C04A90A540EE0A2
:1013D00021460A9800F058F83946009000F054F879
:1013E00025480068425C3046761C04A90A543946F8
:1013F000204600F049F80446002CD6D1314604A816
:10140000FFF7BAFE0AE01099481E0121FFF7B4FE6B
:1014100004E0052119A0FFF7AFFE00BF00BF109840
:101420000078002800D0B7E601900BB0F0BC08BCF3
:1014300004B0184713490870704710B504461148A6
:101440000078002802D02046FFF7A0FE10BD10B59E
:1014500004460C480078012802DD2046FFF796FE7E
:1014600010BD00BFFEE70000348000001005011031
:1014700020000000E0160000E41600004552524F24
:10148000520000001305011030B50B460146002044
:101490002022012409E00D46D5409D4205D31D467A
:1014A0009540491B2546954040191546521E002D72
:1014B000F1DC30BDF8B500242546002904DA0E46DB
:1014C000012400214042B141002B04DA1E460023D2
:1014D00052420125B34100F050F88C4617461E4693
:1014E000AC4203D0002540428D41AC46002C02D0D6
:1014F000002657429E4161463A46334601B0F0BD50
:10150000F0B51FB486B000200090019002900698BC
:10151000069980B204900798090C02040014114344
:1015200007900027089D099806913E463C46039087
:101530000398A9B20204000C039004982D0C1543E3
:1015400048430021224600F048F8C7197141103481
:101550000E46402CECDB3846029A00F03EF8009A2A
:10156000019B80180090594102980191103002901F
:101570004028CCDB00980BB0F0BDF0B51FB4064698
:10158000002082B005464024019100901BE00199A3
:1015900022460F46304600F043F8049A059B801A15
:1015A000994110D310461946224600F016F8361A13
:1015B0008F410197224601200021009F00F00DF885
:1015C00038184D4100902046641E0028DFDC019B46
:1015D00000982946324607B0F0BD10B5202A04DB3A
:1015E0000146203A9140002010BD914020239C1AD2
:1015F0000346E3401943904010BD0000064C01250E
:10160000064E05E0E36807CC2B430C3C98471034AA
:10161000B442F7D3FEF758FD101700003017000052
:1016200010B5202A04DB0846203AD040002110BD26
:101630000B46D340D0402024A21A914008431946BB
:1016400010BD02E008C8121F08C1002AFAD1704775
:101650007047002001E001C1121F002AFBD1704732
:1016600055534152545F496E697400555341525469
:101670005F4465496E69740055534152545F536528
:101680006E64446174610055534152545F52656306
:1016900065697665446174610055534152545F47F2
:1016A00065745278436F756E740055534152545FA0
:1016B0005265616444617461746F42756666005579
:1016C000534152545F53656E644461746146726F56
:1016D0006D42756666004144435F496E697400005F
:1016E000FC160000E816000030313233343536374E
:1016F000383941424344454600000000303132331E
:10170000343536373839616263646566000000003D
:101710003017000000050110140000004216000000
:101720004417000014050110380400005216000090
:1017300000000000000000000000000000000000A9
:04174000010E060090
:04000005000000C136
:00000001FF
